:100000000C9426040C944E040C944E040C944E0450
:100010000C944E040C944E040C944E040C944E0418
:100020000C944E040C944E040C94A5070C941708E1
:100030000C944E040C944E040C944E040C944E04F8
:100040000C944E040C944E040C944E040C944E04E8
:100050000C944E040C944E040C944E040C94060B19
:100060000C944E040C944E040C944E040C944E04C8
:100070000C944E040C944E040C944E040C944E04B8
:100080000C944E040C944E040C944E040C944E04A8
:100090000C94500B0C944E040C944E040C944E048F
:1000A0000C944E040C944E040C944E04F0F89C8E68
:1000B0008783878E9CF8F00000FEFF030303030391
:1000C000070EFCF80000FEFF0303030303070EFC0A
:1000D000F80000FFFF00000000000000FFFF00002C
:1000E000FEFF8383838383C7EE7C380000F8FC0E19
:1000F00007030303070EFCF800003F7FE0C0808089
:10010000C0E07F3FFFFF01010101010101FFFF008E
:1001100000FFFF0C0C0C0C1C3E77E3C100007FFFBE
:10012000C0C0C0C0C0E0703F1F00001F3F70E0C0F3
:10013000C0C0E0703F1F00007FFFC1C1C1C1C1E36B
:10014000773E1C00001F3F70E0C0C0C0E0703F1F42
:10015000000000000001FFFF01000000D5F08D1439
:10016000A1C881CFD9F1AF200043616C656E646591
:1001700072417070004368616E6765204B657973EA
:10018000005361766520262051756974004F6666BC
:10019000004F6E00596561726C793A200044656CBD
:1001A000657465003C20637265617465206E6577D7
:1001B000206E6F7465203E002E0053750053610061
:1001C0004672005468005765005475004D6F004A30
:1001D000616E75617279002046656272756172792F
:1001E000004D6172636800202020417072696C00CC
:1001F0002020204D61690020202020204A756E6556
:1002000000202020204A756C6900202020204175A4
:100210006775737400202053657074656D62657234
:100220004F6B746F62657200204E6F76656D62650C
:100230007200446563656D62657200000000000035
:1002400000000000000000000000000000000000AE
:10025000000000000000000000000000000000801E
:10026000606060606060608000FC02FAFAFAFAFA8E
:10027000FAFAFAEADABA6ADABAFA02FC00806060DC
:10028000606060606080000000000000000000000E
:10029000000000000000000000000000000000005E
:1002A000000000000000000000000000000000004E
:1002B000000000000000000000000000000000003E
:1002C000000000000000000000C03008068382012A
:1002D000315131018283041F20EF2F2F2F2F4F8F99
:1002E0002F8F4F2F2F2E2FEF201F84838201312934
:1002F00031010283060830C0000000000000000049
:1003000000000000000000000000000000000000ED
:1003100000000000000000000000000000000000DD
:1003200000000000000000000000000000000000CD
:10033000000000000000F807182040838201181414
:100340001801C22390C8686FC89622C680BFA0BF9C
:1003500080C62692C86F68C89322C3002810280060
:10036000818241201807F800000000000000000012
:10037000000000000000000000000000000000007D
:10038000000000000000000000000000000000006D
:10039000000000000000000000000000000000005D
:1003A0000000007E010000000000000101814121E9
:1003B0001B04091316161309040304070407040396
:1003C00004091316161309041B2141010101000041
:1003D00000000000017E000000000000000000009E
:1003E000000000000000000000000000000000000D
:1003F000000000FCFCFFFF030303030F0F0C0C00C5
:1004000000FCFCFFFFC3C3C3C3FFFFFCFC0000FFF5
:10041000FFFFFF00080808080404020100FFFFFFB7
:10042000FFC3C3C3C3030303030000FFFFFFFF3C7D
:100430003CF0F0FFFFFFFF0000FFFFFFFF030B0B8F
:1004400003FFFFFCFC0000FCFCFFFFC3C3C3C3FFB2
:10045000FFFCFC0000FFFFFFFFC3C3C3C3FFFF3C63
:100460003C03030F0F0C0C0C0C0F0F030300000FC9
:100470000F0F0F000000000F0F0F0F00000F0F0FE6
:100480000F0C0C0C0C0C0C0C0C00000F0F0F0F0CB5
:100490000C0C0C0C0C0C0C00000F0F0F0F000000CC
:1004A000000F0F0F0F00000F0F0F0F0C0C0C0C03A1
:1004B00003030300000F0F0F0F000000000F0F0FCA
:1004C0000F00000F0F0F0F000003030F0F0C0C4164
:1004D00042434445464748492E2C3F21824A4B4CD3
:1004E0004D4E4F5051522A2F3C3E81535455565732
:1004F00058595A204022282901020408102040801F
:10050000080B0002020201000904000001020200BF
:100510000005240010010524010101042402060540
:1005200024060001070581031000400904010002B0
:100530000A00000007050202400000070583024090
:1005400000000403090412010002EF0201404123EC
:10055000368000010102030141726475696E6F20EB
:100560004C4C430041726475696E6F204C656F6E30
:100570006172646F00000000000000373700000067
:1005800000030700030700123F3F123F12242A3FD7
:100590002A3A122333180633311A3F253F3A2807E7
:1005A00003000000001E3F21000000213F1E00004C
:1005B0000014081400000008083E3E08083818001F
:1005C000000000080808080000303000000000307B
:1005D0003C0F0300001E3F29253F1E223F3F200005
:1005E00000223339292F26113125253F1A0F0F08F4
:1005F0003E3E08173725253D191E3F25253D18018C
:1006000001393D07031A3F25253F1A062F29293FA7
:100610001E3636000000003B1B00000000081C36A0
:1006200022000014141414000022361C08000002DA
:1006300003292D07031E212D2B2F163E3F09093FAD
:100640003E3F3F25253F1A1E3F212133123F3F21C8
:10065000211F1E3F3F292921213F3F090901011E7A
:100660003F212919383F3F08083F3F213F3F2100E4
:10067000001021213F1F013F3F0C1E3B313F3F2017
:100680002020203F270E073F3F3F3F060C3F3F1EE5
:100690003F21213F1E3F3F09090F061E3F21113F09
:1006A0002E3F3F09193F26262725253D1D01013FE5
:1006B0003F01011F3F20203F1F0F1F30301F0F3F02
:1006C0003118303F3F21331E1E3321070F08383FBA
:1006D000072131392D27233F3F21000000030F3C24
:1006E000300000213F3F0000000C0603060C000014
:1006F0000000000000030700000000123A2A2E3E0E
:100700001C3F3F22221E1C1C3E222236141C3C226F
:10071000223F3F1C3E2A2A2E0C043E3F05050006C0
:100720000F29292F1E3F3F02023E3C3D3D20000085
:10073000001020203D1D003F3F181C36221F3F2087
:100740001000003E063C063E3E3E3C04063E3C1C7D
:100750003E22223E1C3E3E12121E0C060F09093F8D
:100760003E3E3E040602002C2E2A2A3A1A023F3F41
:100770002200001E3E20203E1E0E1E30301E0E3E69
:10078000301E303E3E22361C1C3622070F28381FF2
:100790000F2232322A2E26081E3F2100003F3F0042
:1007A000000000213F1E080000180C0C18180C084F
:1007B0001C3E08080E04063F3F060408183F3F1879
:1007C000080C1E3F0C0C0C0C0C0C3F1E0C1C0E07D6
:1007D000070E1C0E1C38381C0E0C1E3F3321000067
:1007E00021333F1E0C0C120C1E041A1E2121212144
:1007F0001E162D392E271B000000000000000000EF
:1008000000000000000000000000000000000000E8
:1008100000000000001F001F1E1F1E1F1F1E1F1EA6
:100820001F6162636465666768692B313233826A6F
:100830006B6C6D6E6F7071722D343536807374759C
:10084000767778797A203D373839191D11241FBE03
:10085000CFEFDAE0DEBFCDBF11E0A0E0B1E0E6ED22
:10086000F1E402C005900D92A03CB107D9F727E052
:10087000A0ECB1E001C01D92A439B207E1F714E089
:10088000C6E2D4E004C02197FE010E94D71EC53203
:10089000D107C9F70E9485130C94E9200C9400003D
:1008A00040913A0250913B02209138023091390236
:1008B00042175307B4F49091E8009570E1F39091DA
:1008C000E80092FD19C08093F10080913A02909166
:1008D0003B0201968F739927892B19F48EEF809331
:1008E000E80080913A0290913B02019690933B027E
:1008F00080933A0281E0089580E00895DF92EF92BC
:10090000FF920F931F93CF93DF93D82E8A017B0121
:10091000E40EF51EEB01CE15DF0571F0D7FE03C026
:10092000FE01849101C088810E94500421968111AA
:10093000F2CF8FEF9FEF01C0C801DF91CF911F91E0
:100940000F91FF90EF90DF900895615030F020916B
:10095000F100FC0120830196F8CF289884E680936B
:1009600082070895CF92DF92EF92FF920F931F9329
:10097000CF93DF936C017A018B01C0E0D0E0CE15FC
:10098000DF0589F0D8016D918D01D601ED91FC91C3
:100990000190F081E02DC6010995892B11F47E01AB
:1009A00002C02196ECCFC701DF91CF911F910F912B
:1009B000FF90EF90DF90CF900895CF93DF931F9239
:1009C000CDB7DEB76983DC01ED91FC910280F38144
:1009D000E02D41E050E0BE016F5F7F4F09950F9021
:1009E000DF91CF91089583E08093E9008091F20038
:1009F000882319F08AE38093E8000895FC01848538
:100A0000958597FD0BC09FB7F89482E08093E9002D
:100A10008091F2009FBF90E0019608959FB7F894EF
:100A200082E08093E9008091F2009FBF90E00895FA
:100A30003FB7F8948091340290913502A09136022C
:100A4000B091370226B5A89B05C02F3F19F001963B
:100A5000A11DB11D3FBFBA2FA92F982F8827820F44
:100A6000911DA11DB11DBC01CD0142E0660F771F94
:100A7000881F991F4A95D1F7089585ED8093BC0092
:100A80008091BC0084FDFCCF10920D02089540912E
:100A9000E701262F30E0240F311D21323105DCF42F
:100AA00020910D022430C9F4FC0180E090E086170B
:100AB00058F43091E7012191DC01AB53BE4FA30FF5
:100AC000B11D2C930196F3CF8091E701680F6093DD
:100AD000E70180E0089581E0089582E00895089597
:100AE0008FEF9FEF08958FEF9FEF08958091C401DE
:100AF00090E09195819591090895CF93DF9300D06F
:100B0000CDB7DEB7CB01642F49835A830E944705D6
:100B10004981842F5A81952F0F900F90DF91CF91AB
:100B20000895CF93DF931F92CDB7DEB7698361E05D
:100B3000CE0101960E94470581E090E00F90DF9181
:100B4000CF9108950895089580E090E008950E945F
:100B5000D4200F931F93CF93DF93EC018881998169
:100B6000009729F02A813B812617370788F48B01EB
:100B70006F5F7F4F0E940A20009761F099838883FE
:100B80001B830A832C813D81232B11F4FC011082ED
:100B900081E001C080E0DF91CF911F910F91089516
:100BA000EF92FF920F931F93CF93DF93FC01248169
:100BB00035816115710511F480E019C041155105A9
:100BC000A9F07B01EC018A01020F131FB8010E94FA
:100BD000A905882389F3288139818C819D81B701FA
:100BE000820F931F0E94E2201D830C8381E0DF911E
:100BF000CF911F910F91FF90EF900895CF93DF93C6
:100C0000EC0188819981009711F00E94721F19826E
:100C100018821D821C821B821A82DF91CF91089557
:100C2000EF92FF920F931F93CF93DF938C017B0181
:100C30006115710569F0FB0101900020E9F731971A
:100C4000EF01C61BD70BBE010E94A905811104C08C
:100C5000C8010E94FE0508C0F801D583C483B7010E
:100C6000808191810E94E220C801DF91CF911F9184
:100C70000F91FF90EF9008950F931F93CF93DF9301
:100C80001F92CDB7DEB782E0898342E450E060E096
:100C900075E080E80E947E040E947113DC011296C8
:100CA0000D911C9113970115110569F0D801ED9173
:100CB000FC910280F381E02DBE016F5F7F4FC80180
:100CC000099597FF07C089810F90DF91CF911F9100
:100CD0000F910895F80100851185E5CF0E946013FA
:100CE00090E008950F931F93CF93DF931F92CDB79A
:100CF000DEB78C01FC018485958597FF0EC0CE017F
:100D000001960E943613019719F4298130E002C040
:100D10002FEF3FEFF80135872487F801848595850B
:100D20000F90DF91CF911F910F910895CF93DF9393
:100D30001F92CDB7DEB7FC018485958597FD05C070
:100D40002FEF3FEF358724870BC0CE0101960E941D
:100D50003613019719F4898190E002C08FEF9FEF5D
:100D60000F90DF91CF910895CF93DF93EC01611540
:100D7000710561F0FB0101900020E9F73197AF01A7
:100D8000461B570B0E94D005811103C0CE010E9463
:100D9000FE05CE01DF91CF910895CF93DF93EC0153
:100DA000FB0144815581608171810E94D0058111D0
:100DB00003C0CE010E94FE05CE01DF91CF910895C0
:100DC000FC01808191810C94721F0F931F93CF932C
:100DD000DF93CDB7DEB761970FB6F894DEBF0FBED5
:100DE000CDBF8C01CB01F8011182108213821282D7
:100DF0001582148250E0BE016F5F7F4F0E94E61D96
:100E0000BE016F5F7F4FC8010E94100661960FB64A
:100E1000F894DEBF0FBECDBFDF91CF911F910F9130
:100E200008950F931F93CF93DF93CDB7DEB76297EB
:100E30000FB6F894DEBF0FBECDBF8C01CB01F80119
:100E400011821082138212821582148250E0BE0138
:100E50006F5F7F4F0E94D01DBE016F5F7F4FC80143
:100E60000E94100662960FB6F894DEBF0FBECDBF8B
:100E7000DF91CF911F910F9108950F931F93CF93FF
:100E8000DF93CDB7DEB729970FB6F894DEBF0FBE5C
:100E9000CDBF8C01862FF80111821082138212823D
:100EA0001582148250E0BE016F5F7F4F90E00E9478
:100EB000E61DBE016F5F7F4FC8010E941006299694
:100EC0000FB6F894DEBF0FBECDBFDF91CF911F915B
:100ED0000F910895EF92FF920F931F93CF93DF939B
:100EE000EC01198218821B821A821D821C826115F4
:100EF000710521F18B01FB0101900020E9F7319789
:100F00007F01E61AF70AB7010E94A905811109C0FD
:100F1000CE01DF91CF911F910F91FF90EF900C9434
:100F2000FE05FD82EC82B80188819981DF91CF9125
:100F30001F910F91FF90EF900C94E220DF91CF91E1
:100F40001F910F91FF90EF9008951F920F920FB68F
:100F50000F9211248F939F938091E1009091E10073
:100F6000937F9093E10083FF0FC01092E90091E01E
:100F70009093EB001092EC0092E39093ED001092AE
:100F8000830798E09093F00082FF20C093E0909355
:100F9000E9009091F200992319F09AE39093E80008
:100FA00090913C02992339F090913C02915090939A
:100FB0003C02992389F190918207992339F090910D
:100FC0008207915090938207992341F184FF10C0CA
:100FD0008091E2008E7E81608093E2008091E1004A
:100FE0008F7E8093E1008091C1018E7E806111C06F
:100FF00080FF16C08091E2008E7E80618093E200C7
:101000008091E1008E7E8093E1008091C1018E7E0F
:1010100081608093C10104C05D9ACDCF289AD6CF5C
:101020009F918F910F900FBE0F901F9018951F9258
:101030000F920FB60F921124CF92DF92EF92FF9290
:101040000F931F932F933F934F935F936F937F93D0
:101050008F939F93AF93BF93EF93FF93CF93DF93C0
:10106000CDB7DEB76C97DEBFCDBF1092E90080919F
:10107000E80083FFEDC168E0CE0145960E94A5041B
:1010800082EF8093E8008D8987FF05C09091E8008A
:1010900090FFFCCF03C09EEF9093E800982F9076CE
:1010A00009F0C6C09E892F89188D91110CC0803817
:1010B00029F48091C2018093F10002C01092F100E6
:1010C0001092F10048C1422F50E0512B913051F461
:1010D000811141C14130510509F03DC18091C201EA
:1010E0008D7F0BC0933061F4811135C141305105C2
:1010F00009F031C18091C20182608093C2012BC18D
:10110000953041F48091E80080FFFCCF2068209367
:10111000E30021C1963009F05FC0EB8CFC8C10928B
:10112000E90010923B0210923A02123091F51092AF
:101130003902109238020E943C0699E0BE016F5FAE
:101140007F4FDB01E92F1D92EA95E9F799831A8316
:1011500091E09E8390EA98879AEF998720913A02CE
:1011600030913B02275F3F4F3C832B838D8310924E
:10117000E90010923B0210923A02F0923902E0929A
:10118000380249E050E080E00E947E040E943C0664
:10119000E2C0F0923902E09238020E947113DC0141
:1011A0001296ED90FC901397E114F10409F4C0C07D
:1011B000D701ED91FC910480F581E02DBE016B5EBD
:1011C0007F4FC7010995009719F00CF0C4C0C7C044
:1011D000F701E084F184E8CF973009F4C0C098307B
:1011E00021F481E08093F100B6C0993009F0B3C0DA
:1011F000837009F0B4C0E4E1F1E081E021E036E37E
:101200009081992361F08093E9002093EB00919104
:101210009093EC003093ED008F5F873089F78EE775
:101220008093EA001092EA008F898093830793C02D
:101230008B8D9C8D1092E90010923B0210923A0225
:101240009093390280933802898D811156C08E891E
:101250009D89913A59F4813209F081C047E050E00C
:1012600065E071E080E00E947E0475C0913209F073
:1012700076C0833289F4888D90E0982F88272F8953
:10128000822BA0E0B0E08093010190930201A09333
:101290000301B09304015FC0803269F48091E800DB
:1012A00082FFFCCF67E085E091E00E94A5048BEF10
:1012B0008093E80006C0823209F04DC08F89809388
:1012C0000C018091C001882319F0EEEFFAE002C012
:1012D000E0E0F8E08091050190910601A0910701FE
:1012E000B0910801803B9440A105B10509F07BC095
:1012F00080910C0180FF93C076C00E947113DC01C5
:1013000012960D911C9113970115110541F1D80109
:10131000ED91FC910190F081E02DBE016B5E7F4F5D
:10132000C8010995811117C0F80100851185ECCF1E
:10133000113009F44EC0133091F48F89882309F4D9
:1013400045C0823081F440E860E184E695E00E9487
:10135000DC1C882321F08EEF8093E80079C081E2C5
:101360008093EB0075C0813029F440E86BE088E59C
:1013700095E0EDCF833099F70E947113DC0112964E
:10138000ED90FC9013978E010F5F1F4F6801E114E1
:10139000F10479F0D701ED91FC910680F781E02D01
:1013A000B801C7010995080F111DF701E084F18408
:1013B000EECFD8011C92F60101900020E9F7319799
:1013C000BF016C197D0940E0C601C1CF62E475E040
:1013D00002C066E475E06115710509F2FB014491F4
:1013E00050E080E840CF0FB6F894A8958091600057
:1013F000886180936000109260000FBEA895EE3F58
:101400002AE0F20739F08091FE0A9091FF0A918359
:101410008083A1CF1092FF0A1092FE0A9CCFEE3F6C
:101420008AE0F80731F0808191819093FF0A8093E0
:10143000FE0A87E797E7918380839BE088E10FB6F8
:10144000F894A895809360000FBE9093600083CFBE
:101450006C960FB6F894DEBF0FBECDBFDF91CF9173
:10146000FF91EF91BF91AF919F918F917F916F917C
:101470005F914F913F912F911F910F91FF90EF90AE
:10148000DF90CF900F900FBE0F901F9018958F9206
:101490009F92AF92BF92CF92DF92EF92FF926B0139
:1014A0007C010E9418054B015C01C114D104E104C8
:1014B000F104F1F00E941805DC01CB0188199909AB
:1014C000AA09BB09883E9340A105B10570F321E04C
:1014D000C21AD108E108F10888EE880E83E0981E50
:1014E000A11CB11CC114D104E104F10419F7DDCF32
:1014F000FF90EF90DF90CF90BF90AF909F908F9034
:1015000008958F929F92AF92BF92CF92DF92EF9207
:10151000FF920F931F93CF93DF935C016B017A01CE
:1015200080910C01882309F45BC080918307882394
:1015300009F456C08091C10180FF05C08091E00090
:1015400082608093E000E70110E00AEF83E0882EDC
:101550009AE3992E2097D9F10E94601381110AC055
:10156000015009F43DC061E070E080E090E00E942D
:10157000470AF0CF282F30E0C217D3070CF48C2F86
:101580004FB7F8948092E9009091E80095FF1DC054
:10159000282F30E0C21BD30BF601982F915020F07A
:1015A00081918093F100FACFC20ED31E112319F05E
:1015B0009092E80009C08091E80085FD06C09092F5
:1015C000E80011E0209709F010E04FBFC3CF1111E0
:1015D000C3CF5D9884E680933C021E141F0444F040
:1015E00081E090E0F5019383828380E090E001C088
:1015F000C701DF91CF911F910F91FF90EF90DF9086
:10160000CF90BF90AF909F908F9008951F920F92B0
:101610000FB60F9211242F933F938F939F93AF9305
:10162000BF938091D1069091D206A091D306B0913C
:10163000D4063091330223E0230F2D3720F4019696
:10164000A11DB11D05C026E8230F0296A11DB11DE5
:10165000209333028093D1069093D206A093D306B1
:10166000B093D4068091340290913502A091360255
:10167000B09137020196A11DB11D80933402909361
:101680003502A0933602B0933702BF91AF919F917C
:101690008F913F912F910F900FBE0F901F90189533
:1016A0001F920F920FB60F9211242F933F934F93D7
:1016B0005F936F937F938F939F93AF93BF93EF93BA
:1016C000FF938091B900887F803609F49CC068F54B
:1016D000883209F45BC090F4803109F454C038F4C6
:1016E000882309F4F6C0883009F44DC0F6C088316B
:1016F00009F44CC0803209F45DC0EFC0803409F4B5
:1017000068C048F4803309F455C0883309F0E5C057
:1017100080930C02D8C0803509F44FC0883509F495
:101720005DC0883409F0D9C0D6C0883909F4C7C073
:10173000A8F4883709F467C038F4883609F463C020
:10174000803709F460C0C9C0883809F4B8C080394E
:1017500009F45FC0803809F0C0C05BC0803B09F469
:1017600086C038F4803A09F466C0883A09F47FC02C
:10177000B4C0803C09F4A7C0883C09F4A4C0883BED
:1017800009F48AC0AAC08091320210C0909131023F
:1017900080913002981770F5E091310281E08E0F50
:1017A00080933102F0E0E05FFD4F80818093BB00C9
:1017B00085EC86C080930C028EC0E091310281E0FE
:1017C0008E0F809331028091BB00F0E0E05FFD4F0F
:1017D000808390913102809130026EC0E09131029D
:1017E00081E08E0F809331028091BB00F0E0E05FDA
:1017F000FD4F808380910F0281116DC081E0809345
:101800000E0284EA61C083E080930D0210920B0205
:10181000CFCF80910B02803208F051C0E0910B02D3
:1018200081E08E0F80930B028091BB00F0E0E551C8
:10183000FE4F8083BDCF85EC8093BC0010920D02DB
:1018400080910B02803230F4E0910B02F0E0E55120
:10185000FE4F108260910B0270E0E091E901F0917F
:10186000EA018BEE91E0099510920B0236C084E0FC
:1018700080930D021092E8011092E701E091E501DA
:10188000F091E60109958091E701811105C081E0A1
:101890008093E7011092C501E091E80181E08E0F8D
:1018A0008093E801F0E0EB53FE4F80818093BB0012
:1018B0009091E8018091E701981708F479CF85E8C5
:1018C0008093BC000AC085EC8093BC0010920D028E
:1018D00004C010920C020E943D05FF91EF91BF9150
:1018E000AF919F918F917F916F915F914F913F91B8
:1018F0002F910F900FBE0F901F9018952D9A08955D
:10190000BC0180E090E00C94470A8FB18095807F05
:10191000669B88601C9B8460089560387105D0F4D4
:1019200040345105B8F4E8EFF4E080E1849FD00141
:10193000A0781124A60F4770E40FF11D8491A35CD9
:10194000BD4F222319F06C91862B03C080956C91BA
:1019500086238C930895982F9F7D99F0805280372D
:1019600008F08FE396E0899FF0011124E658FA4FC2
:1019700086E09491911106C0815031978111F9CF81
:10198000089586E008950C941B1EFC017383628306
:10199000808191816817790741F08617970714F4C1
:1019A000019601C001979183808357834683848188
:1019B00095814817590741F08417950714F401964B
:1019C00001C00197958384830895EF92FF920F934E
:1019D0001F93CF93DF931F92CDB7DEB77C01FC013D
:1019E00000811181C80169830E941B1E69816817EB
:1019F00019F0C8010E94231EC7010F90DF91CF91FB
:101A00001F910F91FF90EF900895CF93DF93209156
:101A1000480630E08091440660914B0670914C0678
:101A2000681B710940E051E0842F90E028173907C6
:101A3000ACF0EC01C60FD71FFC01EF54F94F108238
:101A4000ADE4B6E08D919D918C179D0709F450830C
:101A500086E0A13BB807B1F74F5FE6CFDF91CF91AA
:101A6000089540914606509147069A01205D3740FF
:101A70006DE671E0269FC001279F900D369F900D67
:101A8000112437FF02C02D5F3F4F359527953595BF
:101A90002795820F931F9A01237033275091450693
:101AA0002115310511F4523008F0019665E178E016
:101AB000FB014E2F461B451770F4413029F42115C8
:101AC000310521F04CE103C0449101C04DE1840F88
:101AD000911D3196EECF20914406820F911D909377
:101AE0004C0680934B060895E091D906F091DA06F2
:101AF0000280F381E02D42E050E062E671E089ED82
:101B000096E009948F929F92AF92BF92CF92DF920C
:101B1000EF92FF920F93CF93DF936B01EC014C0197
:101B2000840E911C5B01A20EB11CC815D905ECF402
:101B30007601D7FE10C0E12CF12C0DC0E816F90695
:101B400094F4202FA701BE018BE697E00E948D0C34
:101B50002FEFE21AF20AC50121E4A216B10474F3D0
:101B600080E490E0EBCF2196E0CFDF91CF910F9111
:101B7000FF90EF90DF90CF90BF90AF909F908F90AD
:101B80000895811102C080E008958FB7F8944091C4
:101B9000D1065091D2066091D3067091D4068FBFC2
:101BA0008091D5069091D606A091D706B091D8061F
:101BB000481759076A077B0730F32FB7F8948091CD
:101BC000D1069091D206A091D306B091D4062FBF32
:101BD00088539F4FAF4FBF4F8093D5069093D60643
:101BE000A093D706B093D80681E00895CF93DF93F2
:101BF000E091D906F091DA06DC0114964D915C91E2
:101C000015976D917C910280F381E02D89ED96E02E
:101C10000995EC010E94740D8C0F9D1FDF91CF91EF
:101C200008954F925F926F927F928F929F92AF92A0
:101C3000BF92CF92DF92EF92FF920F931F93CF93B9
:101C4000DF93CDB7DEB762970FB6F894DEBF0FBE55
:101C5000CDBFE091D906F091DA060280F381E02D44
:101C60004BE050E065E671E089ED96E009950E9451
:101C7000740D3DE4E32E36E0F32E4701612C712C08
:101C800010E086E590E09C0129523740590184E537
:101C900097E002E1080FF401219131914F01809109
:101CA0004B0690914C062817390709F04AC04AE0C4
:101CB000612FCE0101960E943D0760914B06709105
:101CC0004C064AE0CE0107960E94E50661E771E006
:101CD000CE010D960E946A07BE01695F7F4FCE015B
:101CE0000D960E94CD066BE771E00E94B406BE011E
:101CF0006F5F7F4F0E94CD060E94F60DCE010D96BC
:101D00000E94E006CE0107960E94E006CE010196F1
:101D10000E94E00624E5C22E27E0D22E2501460CC3
:101D2000571CF60161916F01C2018E0F9F1F9A83AC
:101D30008983CE0101960E94E50C0C11F2CF81E05F
:101D400001C080E01F5F123309F444C0F2E16F0E5E
:101D5000711C882309F49FCF0E94050D60914406F1
:101D600080E190E09A838983CE0101960E94E50C80
:101D70006091450681E190E09A838983CE010196C6
:101D80000E94E50C60914606605D82E190E09A83D6
:101D90008983CE0101960E94E50C83E090E0909348
:101DA00043068093420662960FB6F894DEBF0FBEDC
:101DB000CDBFDF91CF911F910F91FF90EF90DF90FA
:101DC000CF90BF90AF909F908F907F906F905F90DB
:101DD0004F9008958111C0CF0EE110E0812C912C1D
:101DE000712C86E590E09C0129523740590184E529
:101DF00097E092E1692E680EF70180819181892B2D
:101E000009F063C04AE0672DCE0101960E943D07AC
:101E100060914B0670914C064AE0CE0107960E94F5
:101E2000E50661E771E0CE010D960E946A07BE01EA
:101E3000695F7F4FCE010D960E94CD0666E971E085
:101E40000E94B406BE016F5F7F4F0E94CD060E94C4
:101E5000F60DCE010D960E94E006CE0107960E9477
:101E6000E006CE0101960E94E00680914B0690911B
:101E70004C068F839887F70180839183682F1A839C
:101E80000983CE0101960E94E50C6885C801019680
:101E90009A838983CE0101960E94E50C84E5C82EC1
:101EA00087E0D82E2501480C591CF60161916F017D
:101EB000C2018E0F9F1F9A838983CE0101960E94D3
:101EC000E50C6C10F2CF81E001C080E07394003823
:101ED000110509F441CFF2E0EF0EF11C22E1820E70
:101EE000911C0E5F1F4F882309F486CF35CF2091B8
:101EF0007107282329F490917007982381E009F451
:101F000080E008950E94310D80914B0690914C061F
:101F1000059620914406821B910967E070E00E94BB
:101F2000C31E80934906E0914506E13051F42091AB
:101F300046063091470623703327232B39F0ECE116
:101F400006C0F0E0EB5EF74FE49101C0EDE1E093F5
:101F50004806EE3110F485E005C0EE3139F40697FD
:101F6000D1F786E080934A060C94050D85508230A7
:101F700090F7F7CF8091440690914806891728F48E
:101F80008F5F809344060C94310D81E0809344066A
:101F9000809145068A3020F48F5F809345060BC000
:101FA00010924506809146069091470601969093BF
:101FB0004706809346060C94820F80914406823037
:101FC00028F08150809344060C94310D8091450691
:101FD000882321F081508093450610C08BE08093C8
:101FE00045068091460690914706813D27E092077D
:101FF00028F0019790934706809346060E94820F2F
:1020000080914806809344060895EF92FF920F93C3
:102010001F93CF93DF93CDB7DEB768970FB6F894D1
:10202000DEBF0FBECDBF082F162F7A014AE0B701E1
:10203000CE0101960E941107612F012E000C770B33
:102040004AE0CE0107960E941107602F002E000C77
:10205000770B4AE0CE010D960E9411076DEA71E000
:10206000CE0143960E946A07BE01635F7F4FCE0197
:1020700043960E94CD066DEB71E00E94B406BE014E
:10208000695F7F4F0E94CD066DEB71E00E94B40640
:10209000BE016F5F7F4F0E94CD060E94F60DCE01FC
:1020A00043960E94E006CE010D960E94E006CE0106
:1020B00007960E94E006CE0101960E94E0061F3FAF
:1020C00021F48BE08093450607C01C3019F4109270
:1020D000450602C01093450680EDE81687E0F80635
:1020E0003CF480ED97E0909347068093460604C049
:1020F000F0924706E0924606009344060E94820F43
:102100008091480690914406891710F48093440604
:1021100068960FB6F894DEBF0FBECDBFDF91CF91AA
:102120001F910F91FF90EF9008955F926F927F92B1
:102130008F929F92AF92BF92CF92DF92EF92FF92D7
:102140000F931F93CF93DF9320913D0630913E066E
:102150002A5F3F4F2738310508F0BFC020913F0666
:1021600030914006A901495F5F4F4834510508F09E
:10217000B4C0873609F4A8C0982F977F913709F427
:10218000A3C0612CC82F0E94AB0C7090410690EE4A
:102190009C0F903708F09FE360913F0670914006D6
:1021A000C0913D06D0913E069B01285F3F4F482FCE
:1021B00050E02934310550F0662009F47CC06150AC
:1021C00071097093400660933F0675C09E01240F0D
:1021D000351F37FDF1CFC138D10574F77B0187E09A
:1021E000E822FF244B0177FF03C0A7E08A0E911C71
:1021F00083E0959487948A95E1F79694982C8824A7
:1022000097948794F6E09F9F50011124CE01AC1A59
:10221000BD0A08E010E00E191F099C012C1B3D0BA4
:102220002417350748F6F501E80FF91FEB58FA4F68
:10223000E4919C01280D391D2115A4E03A07C8F549
:1022400080389105B0F5D901A35CBD4FF0E077FD72
:1022500021C071100AC06F010E2C01C0CC0C0A9471
:10226000EAF7C094DC90CD2008C05C906F010E2C82
:1022700001C0CC0C0A94EAF7C528CC92E114F10411
:10228000C1F02038A3E03A07A4F420583F4FD90109
:10229000A35CBD4F002E02C0F595E7950A94E2F7C6
:1022A000711004C0E0952C91E22302C02C91E22B26
:1022B000EC930196B2CF4F5F5F4FC40FD51FD09301
:1022C0003E06C0933D0609C02F5F3F4F3093400646
:1022D00020933F066624639455CFDF91CF911F91E1
:1022E0000F91FF90EF90DF90CF90BF90AF909F90B5
:1022F0008F907F906F905F900895CF92DF92EF92D2
:10230000FF920F931F93CF93DF936C01649F700133
:102310001124C42FD0E000E010E00C171D0769F075
:10232000F801EE0DFF1DEC0DFD1D84910F5F1F4F99
:10233000882319F00E949510F0CFDF91CF911F9163
:102340000F91FF90EF90DF90CF9008954F925F92A2
:102350006F927F928F929F92AF92BF92CF92DF92B5
:10236000EF92FF920F931F93CF93DF934B015C018A
:1023700097FF08C0B094A09490948094811C911C05
:10238000A11CB11C2401350110E0C12CD12C760117
:10239000C3944114510461047104C1F01F5FC3016F
:1023A000B2012AE030E040E050E00E94311E2901F5
:1023B0003A01232B242B252B61F3AAE0B0E0A701DF
:1023C00096010E94501E6B017C01E3CF00E0CAE041
:1023D000D0E08AE0482E512C612C712C0117B9F005
:1023E000C501B401A70196010E94311EC901BE01B9
:1023F0000E94C31E805D0E949510C701B601A30113
:1024000092010E94311E69017A010F5FE7CFDF91CF
:10241000CF911F910F91FF90EF90DF90CF90BF90E1
:10242000AF909F908F907F906F905F904F900895A6
:102430001F93CF93DF93EC01FE011491812F0E9433
:10244000951021961111F8CFDF91CF911F9108952A
:102450002F923F924F925F926F927F928F929F92B4
:10246000AF92BF92CF92DF92EF92FF920F931F93A2
:10247000CF93DF93CDB7DEB728970FB6F894DEBFC2
:102480000FBECDBF5A01822E912C9C01280D391D03
:1024900037FDC4C0803891050CF0C0C09B01200FEF
:1024A000311D37FDBBC0603471050CF0B7C0AB0106
:1024B00077FF04C044275527461B570B4770552705
:1024C0009B0177FF02C0295F3F4FE3E035952795D9
:1024D000EA95E1F777FF08C02150310968E070E024
:1024E000DB01A41BB50BAD01602F66956695669563
:1024F00070E0077011F06F5F7F4FDB01A20FB31F19
:10250000BA83A98339017694762C662477946794EC
:10251000680E791EE12CF12C00E010E02301B0E8F8
:102520004B0E511C68E070E0DB01A41BB50BBC83B3
:10253000AB8369817A812617370709F46FC0283089
:10254000310509F46BC02F3FBFEF3B070CF45BC0B4
:10255000B201600F711FDB01A35CBD4FBE83AD8371
:10256000D801A60DB71DA35CBD4F6C0160E070E003
:10257000681579050CF047C0E0E8CE16D10409F4DF
:1025800042C0D7FC34C02F3FFFEF3F0709F442C0E1
:10259000FB01EE0DFF1DEA0DFB1DE491042E01C0B1
:1025A000EE0F0A94EAF73C90E329EC9341155105AC
:1025B000F1F027303105D9F0FB01EE0DFF1DEA0DDA
:1025C000FB1DE4912E2E312CF1010B8002C0F595FC
:1025D000E7950A94E2F7F887EF83ED81FE8130807A
:1025E000EF81F885E3291F01ED81FE8120826F5F75
:1025F0007F4FED81FE813196FE83ED83FFEFCF1A91
:10260000DF0A1196B5CF2F5F3F4F00581F4FE80CE0
:10261000F91C8FCF4115510579F6E9CF28960FB6F1
:10262000F894DEBF0FBECDBFDF91CF911F910F9108
:10263000FF90EF90DF90CF90BF90AF909F908F90E2
:102640007F906F905F904F903F902F900895EDE3B3
:10265000F2E0A0E0B8E000800EBC8111012C1197DF
:10266000A0FDFDCF0192B9F70DB40895FC01809152
:102670008307811103C08FEF9FEF08959FB7F894F0
:1026800082E08093E9002091F20030E012161306F8
:1026900014F421E030E02115310559F0289884E642
:1026A000809382078091F10080838091F2008823DB
:1026B00019F09FBFC90108958BE68093E800F9CF18
:1026C0002FB7F89483E08093E9009091E800892F78
:1026D000807295FF04C09091F20080E4891B2FBFA7
:1026E00008958091880781110DC082E0809384074E
:1026F00084E080938507109287071092860781E017
:102700008093880784E897E00895CF93DF93CDB74F
:10271000DEB76A970FB6F894DEBF0FBECDBF7894D0
:1027200084B5826084BD84B5816084BD85B58260D6
:1027300085BD85B5816085BD80916E008160809387
:102740006E001092810080918100826080938100F0
:102750008091810081608093810080918000816000
:10276000809380008091910082608093910080919D
:1027700091008160809391008091900081608093AE
:1027800090008091C10084608093C1008091C1005D
:1027900082608093C1008091C10081608093C100FC
:1027A0008091C30081608093C3008091C0008260EB
:1027B0008093C0008091C20081608093C2008091AC
:1027C0007A00846080937A0080917A00826080939E
:1027D0007A0080917A00816080937A0080917A00FB
:1027E000806880937A00109283071092C201109241
:1027F000C1018091D70081608093D70080EA8093E7
:10280000D80089B5806189BD89B5826089BD09B468
:1028100000FEFDCF61E070E080E090E00E94470A9A
:102820008091D8008F7C80618093D8008091E000F7
:10283000807F8093E0008091E1008E7E8093E100B4
:102840008DE08093E200559A209AEEEFFFE78591A4
:1028500094918B3F9C4D19F481E08093C0018FEFE0
:102860009FEF9093E6068093E50664E670E080E0D3
:1028700090E00E94470A80E18093720781EC809388
:102880007C0085B1806F85B984B1877E84B984B1BD
:10289000876E84B95E9A5F988AB1806D8AB9769A9C
:1028A0006E9881B3806F81BB899880B38D7080BB37
:1028B00080E58CBD81E08DBD85E090E00E94800CBC
:1028C0005F9A85E090E00E94800C5E985C98ECE551
:1028D000F1E08DE08E0F94919EBD00000DB407FED7
:1028E000FDCF31968E13F7CF5C9A81E88093640018
:1028F0008091650081608093650080E00E942713CD
:102900000E94850C87FF16C05C9885EA8EBD00008A
:102910000DB407FEFDCF8EB55C9A2E982F982D989A
:102920008091640080628093640081E083BF889519
:1029300013BEFCCF02E010E00E94850C82FF42C073
:102940002D980E94850C84788438C9F00E94850CEB
:102950008471843191F50E947E0C88EC90E00E9495
:10296000800C2E981A83098360E0CE0101960E94A4
:10297000E50C84EF91E00E94800C2E9A19C00E9411
:102980007E0C88EC90E00E94800C2F981A830983BB
:102990006FEFCE0101960E94E50C84EF91E00E945A
:1029A000800C2F9A0E94850C84788438D9F3CECF7E
:1029B0000E94850C84718431D9F388EC90E00E94E8
:1029C000800CBACF0E947E0C82E090E00E941B1E19
:1029D000882329F03E9A3F9A81E08093C30181E0E9
:1029E00090E00E941B1E82FB112710F981E090E00D
:1029F0000E941B1E81FF3AC011112E98B0EFEB2EE2
:102A0000FF24FA940E94850C86FF04C02E9A2F9A08
:102A10002D9A2CC0112331F034E0E316F10411F4A7
:102A20002E9A2F9881E00E94271300E128E54CEAB6
:102A300050E0B70184E190E00E94281280E00E94FB
:102A400027138FE090E00E94800C8FEFE81AF80ABD
:102A500099E1E916F104B1F6112311F02F9A2D989E
:102A600080E991E00E94800C0E947E0C82E390E05D
:102A70000E94800C0E94850C8111F8CF81E0809328
:102A8000000103E110E0C8010E94C30CF801EA5AFA
:102A9000FE4FE4918E13109200010F5F1F4F0E3115
:102AA000110589F7809100018823E9F080910001E8
:102AB000882309F43FC080E190E00E94C30C80931A
:102AC000440681E190E00E94C30C8093450682E1B8
:102AD00090E00E94C30C90E08053984F909347067B
:102AE000809346062DC0A0E1EA2EF12CFA82E982FD
:102AF00060E0CE0101960E94E50CEFEFEE1AFE0AAF
:102B0000F0E1EF16F4E0FF0689F7F3E1EF2EF12C88
:102B1000F701EA5AFE4F6491FA82E982CE010196EA
:102B20000E94E50C2FEFE21AF20A3EE1E316F104EF
:102B300079F7BCCF43EE57E06AE081E00E940510D0
:102B40001092430610924206EDE4EE2EE6E0FE2ED1
:102B5000C8010E941B1E8983C80101960E941B1E8A
:102B60008A8389819A81F701819391937F010E5F16
:102B70001F4F0238110561F780910001811138C0A3
:102B800081E48093540782E78093550784E680931D
:102B9000560785E78093570782E6809358078FE6AC
:102BA0008093590789E780935A0780E280935B07F7
:102BB00097E490935C0721E620935D079DE6909350
:102BC0005E0735E630935F07809360073AE4309301
:102BD000610720936207909363078093640784E3FF
:102BE000809365070E94110E1092430610924206D0
:102BF0000E94820F87E590E09C0129523740388F70
:102C00002F8B8FB7F8944091D1065091D2066091E6
:102C1000D3067091D4068FBF80917307942F981BB1
:102C200080917407882329F0909375071092740798
:102C3000B4C620917207921748F49F5F921708F06C
:102C4000ACC681E083BF889513BEA7C611E0109380
:102C500074074093730720916E0730916F072F5FC1
:102C60003F4F30936F0720936E07EDE3F2E0811141
:102C70008FEF002481938193819381930394D1F703
:102C800080917007809371070E94850C8093700774
:102C900080914206909143068230910509F403C168
:102CA0002CF4009759F0019791F0EDC28330910513
:102CB00009F4A2C1049709F4CBC1E5C288E00E94DF
:102CC000770F882309F4DFC281E090E0E7C020910C
:102CD0003D0730913E0780913F07909140072817AC
:102CE000390771F5109341060E94850C85FF03C0DA
:102CF00081E590E002C082E590E090933E068093EB
:102D00003D068BE090E09093400680933F0686E876
:102D10000E9495100E94850C86FF03C089E790E011
:102D200002C088E790E090933E0680933D068BE0DA
:102D300090E09093400680933F0687E80E949510AC
:102D400020913507309136078091370790913807E9
:102D500028173907D9F581E0809341060E94850C38
:102D600087FF09C08CE190E090933E0680933D067A
:102D700083E090E008C08CE190E090933E06809361
:102D80003D0684E090E09093400680933F0684E8FF
:102D90000E9495100E94850C84FF09C08CE190E090
:102DA00090933E0680933D0682E190E008C08CE15E
:102DB00090E090933E0680933D0683E190E09093EF
:102DC000400680933F0685E80E9495100E94850C7E
:102DD00091E084FF90E0892F0E94C10D882359F073
:102DE0004091460650914706609145066F5F80917D
:102DF00044060E9405100E94850C982F991F992760
:102E0000991F892F0E94C10D882359F040914606D1
:102E100050914706609145066150809144060E949A
:102E200005100E94850C91E086FF90E0892F0E949A
:102E3000C10D882361F040914606509147064F5FCF
:102E40005F4F60914506809144060E9405100E94E4
:102E5000850C91E085FF90E0892F0E94C10D8823A9
:102E600061F04091460650914706415051096091EA
:102E70004506809144060E94051084E00E94770F69
:102E8000882321F0109243061092420688E00E94A7
:102E9000770F882309F4F7C182E090E0909343060E
:102EA00080934206F0C180E20E94770F81110E9458
:102EB000DD0F80E40E94770F81110E94BA0F80E835
:102EC0000E94770F811106C080E10E94770F811167
:102ED00007C00BC017E00E94DD0F1150E1F7F4CFDF
:102EE00017E00E94BA0F1150E1F784E00E94770FBB
:102EF000882331F081E090E090934306809342066E
:102F000088E00E94770F882309F4BDC183E090E038
:102F100090934306809342067DE4C72E76E0D72E39
:102F2000E12CF12C80E010E024E537E002E1020F13
:102F3000F601419151916F0120914B0630914C0661
:102F40004217530709F046C04AE0612FCE010D96A3
:102F50000E943D0760914B0670914C064AE0CE01FD
:102F600007960E94E50664E471E0CE0101960E9496
:102F70006A07BE01695F7F4FCE0101960E94CD06B0
:102F800060E571E00E94B406BE01635F7F4F0E945E
:102F9000CD060E94F60DCE0101960E94E006CE01FC
:102FA00007960E94E006CE010D960E94E00664E5B9
:102FB000862E67E0962EAF88B88CAE0CBF1CC5017C
:102FC000880D991D0E94C30CF40181934F010E13CB
:102FD000F6CF81E01F5FF2E1EF0EF11C123309F032
:102FE000A7CF811150C1E4E5F7E090E282E18E0FB6
:102FF00091938E13FDCF47C184E00E94770F81111A
:10300000D4C480E80E94770F8111CFC480E10E9470
:10301000770F8111CAC480E20E94770F8111C5C465
:1030200080E40E94770F8111C0C488E00E94770F6E
:10303000882309F428C184E090E0909343068093AC
:1030400042061092530710925107109252071BC16B
:1030500084E00E94770F882331F083E090E0909322
:1030600043068093420688E00E94770F882309F484
:1030700087C080916807882309F47CC0E0915107DC
:1030800080915207ED3009F044C0811123C0909126
:103090006A0780915307992339F0E82FF0E0EC5C40
:1030A000F84F90E290A311C0982F882309F468C0CC
:1030B000923140F4E92FF0E0E75DF84F23A522A715
:1030C0009F5FF6CF90E290936507882309F458C07C
:1030D00081504DC0813089F48091660790916707D7
:1030E0008152984019F48FEC94E002C081E298E09C
:1030F000909367078093660743C0823039F49091BC
:10310000690781E08927809369073AC00E94110E00
:1031100037C0F0E03EE0839FE00DF11D1124809167
:10312000660790916707E80FF91F449180916A073D
:10313000882361F080915307A82FB0E0AC5CB84FB2
:1031400090964C938131E0F48F5F11C090915307BA
:10315000A5E6B7E080E18A1B282F2A0F921750F7C7
:103160009D0122503109F90120812E93F5CF8093E2
:10317000530706C090916A0781E0892780936A0708
:103180000E94850C91E084FF90E0892F0E94C10D80
:103190008823A1F080916807882369F08091520705
:1031A000833060F48F5F80935207833039F48DE071
:1031B0008093510703C081E0809368070E94850CCB
:1031C000982F991F9927991F892F0E94C10D882335
:1031D00099F080916807882379F0809152078823BD
:1031E00049F0833019F49DE090935107815080930A
:1031F000520702C0109268070E94850C91E086FF7A
:1032000090E0892F0E94C10D8823D1F0809168073A
:10321000882379F080915207833091F08091510793
:103220008D3020F48F5F809351070AC010925107B0
:1032300007C080915307813118F48F5F8093530743
:103240000E94850C91E085FF90E0892F0E94C10DBE
:103250008823C9F080916807882371F08091520714
:10326000833089F080915107882311F0815001C08B
:103270008DE08093510707C080915307882319F090
:103280008150809353078091420690914306892B89
:1032900019F440E050E002C04EEC5FEF69E070E0EE
:1032A00089E297E00E94C50C60912D0770912E076E
:1032B0000CE22EE64BE352E08091290790912A0719
:1032C0000E9428128091420690914306009729F4AB
:1032D00042E350E063E170E011C08130910529F4D0
:1032E0004BE050E06EE070E009C0029719F440E056
:1032F00050E002C046EF5FEF63E070E089E397E0E3
:103300000E94C50C81E08093410680913D07909119
:103310003E072091390730913A0730933E062093BB
:103320003D069093400680933F0649E06091450634
:103330008FEC91E00E947D118091420690914306AE
:10334000009729F442E350E063E570E011C081305A
:10335000910529F44BE050E06BE570E009C002975D
:1033600019F440E050E002C046EF5FEF63E670E022
:1033700081E397E00E94C50C81E080934106809133
:1033800035079091360720913107309132073093FD
:103390003E0620933D069093400680933F06609141
:1033A00046067091470680E090E00E94A611809149
:1033B000420690914306009719F440E450E013C090
:1033C0008130910519F44CE150E00DC08230910537
:1033D00019F448E050E007C0039719F440EF5FEF9D
:1033E00002C040EC5FEF60E070E081E497E00E9493
:1033F000C50C81E08093410653E0E52EF12C10E0EE
:1034000080914507909146070196F0923E06E09222
:103410003D069093400680933F06111103C08CEC4B
:1034200091E01BC0113019F489EC91E016C0123004
:1034300019F486EC91E011C0133019F483EC91E09B
:103440000CC0143019F480EC91E007C0153019F469
:103450008DEB91E002C08AEB91E00E9418121F5F91
:10346000F2E1EF0EF11C173059F6E090490630906A
:10347000480680914A06863018F038E019E002C00C
:1034800039E01AE0109241066091450770914607B5
:10349000685F7F4F01E020E340E880E090E0398FF3
:1034A0000E94820DA12CB12C398D832F90E09E8B30
:1034B0008D8BC12ED12C2224239480914A0690E03A
:1034C000A816B9060CF0B5C04E2C512CED89FE891A
:1034D000AE9E4001AF9E900CBE9E900C1124F2E176
:1034E000EF9E70011124F7E04F1651040CF09CC0C0
:1034F000332009F499C03A94109148061319812F8A
:1035000090E000E03C016AE070E00E94C31E805D34
:10351000698F7A8F0E94AB0C90E09C01200F311DC7
:10352000698D862F7A8D972F009719F001E0020F91
:10353000EACF8EE090E0821B910997FD01969C01F5
:10354000359527953C8B2B8B80914406181313C01F
:103550002092410660914507709146076C0D7D1DD4
:1035600061507109680D791D00E028E041E1C70153
:1035700001960E94820DF301EF54F94F8081882358
:1035800051F131E080914406181330E06091450715
:10359000709146076C0D7D1D61507109680D791D94
:1035A000032F22E042E0370180E1680E711CC30165
:1035B000398F0E94820D398D21E0232740914507E4
:1035C000509146074C0D5D1D480D591DB3018BE60A
:1035D00097E00E948D0C80914507909146078C0DD5
:1035E0009D1D880D991D2B893C892D5F3F4F2E0D08
:1035F0003F1D30933E0620933D06909340068093F6
:103600003F06612F70E080E090E00E94A61180915B
:103610004406181302C0109241069FEF491A590A36
:10362000E2E1EE0EF11C5FCF2FEFA21AB20AE12CFD
:1036300044CF80914206909143068330910519F45E
:103640004AE250E007C0049719F440E050E002C09D
:1036500042E450E060E070E089E497E00E94C50C2D
:1036600060914D0770914E076A5E7F4F01E02CE23A
:1036700040E880E090E00E94820D81E08093410666
:1036800080914D0790914E07029620914907309105
:103690004A07265F3F4F30933E0620933D069093A6
:1036A000400680933F066091440670E080E090E021
:1036B0000E94A61188EB91E00E94181249E06091E7
:1036C00045068FEC91E00E947D1180E20E949510EA
:1036D000609146067091470680E090E00E94A61136
:1036E0008AE30E94951080916E0780FF34C080911C
:1036F000420690914306049771F524E5E22E27E0F7
:10370000F22E10E000E0F70181917F010E94AB0CE6
:1037100090915307901741F0E12FE80F11E01E0F31
:103720000F5F023181F780E090916A0760914D0749
:1037300070914E07E12FF0E0645F7F4F01E028E0D9
:10374000992321F0482FCF01039603C041E0CF0118
:1037500002960E94820D81E08093410680914D0780
:1037600090914E070D9623E030E030933E06209373
:103770003D069093400680933F06809142069091CB
:103780004306039769F4E0914406F0E0EF54F94FE3
:103790008081811105C084EA91E00E9418120CC05A
:1037A00004E517E092E1F92EF00EF80181918F0106
:1037B0000E949510F012F9CF1092410610E0A12C52
:1037C000B12C812C912C7724739483E0C82ED12CBA
:1037D000E12CF12C8091510790E0E816F906D9F41C
:1037E0008091520790E088169906A9F480916807A5
:1037F000882389F07092410660914D0770914E07C1
:10380000655E7F4F6A0D7B1D00E028E04AE0C6013F
:1038100002970E94820D80914D0790914E074C9621
:103820008A0D9B1DD0923E06C0923D0690934006A5
:1038300080933F0641E0612F6E0D80916607909165
:1038400067070E947D1120915107822F90E0E816B2
:10385000F90641F48091520790E08816990611F418
:1038600010924106FFEFEF1AFF0A39E0C30ED11C98
:103870008EE0E816F10409F0ADCF9FEF891A990A9E
:10388000E9E0AE0EB11C125F1A3209F09ECF8091B2
:103890004D0790914E078E9648E750E050933E06B4
:1038A00040933D069093400680933F062D3041F4AF
:1038B00080915207823021F481E08093410602C05A
:1038C0001092410680916907882311F08AE801C0AF
:1038D00089E80E94951060914D0770914E0788E726
:1038E00090E090933E0680933D06CB01C79690935F
:1038F000400680933F0680915207833089F480917F
:103900006807882349F06A5C7F4F00E028E04AE0BE
:1039100086E790E00E94820D81E08093410602C01C
:103920001092410688E80E94951080914D07909171
:103930004E07C99623E030E030933E0620933D06C3
:103940009093400680933F06109241068091510764
:103950008D3001F580915207811103C08DE991E00E
:1039600017C0813019F485E791E012C0823071F4FC
:1039700084E991E00E94181280916907882319F068
:1039800081E991E005C08DE891E002C081E891E015
:103990000E94181280E00E94271380E090E0892B9B
:1039A00009F42FC90E9400002CC982E090E0909396
:1039B00043068093420639CBCF92DF92EF92FF927B
:1039C0000F931F93CF93DF931F92CDB7DEB7182FBE
:1039D000062FE42E862F880F8E5F99830E94500455
:1039E00083E00E945004F12EC12E9981D92E8C2D96
:1039F0008F19801798F4F601E7FE02C0849101C088
:103A000080810E945004182F80E00E94500481237E
:103A1000FFEFCF1ADF0A8111EACF01C081E00F90DA
:103A2000DF91CF911F910F91FF90EF90DF90CF909A
:103A300008951092DC061092DB0688EE93E0A0E079
:103A4000B0E08093DD069093DE06A093DF06B0938E
:103A5000E0062EE131E03093DA062093D9062FEF0D
:103A60003FEF3093E6062093E50610927907109217
:103A7000780780937A0790937B07A0937C07B09395
:103A80007D0780E391E0909377078093760782E447
:103A900091E090936C0780936B07109270071092DF
:103AA000710780E18093720710926F0710926E0782
:103AB00010927407109251071092520710925307F8
:103AC00081E08093680781E298E090936707809394
:103AD000660710926A07E4E5F7E090E282E18E0F54
:103AE00091938E13FDCF89E090E090932A07809305
:103AF000290790932C0780932B0710922E07109282
:103B00002D071092300710922F0783E190E09093D9
:103B10003A078093390790933C0780933B0782E3F1
:103B200090E090933E0780933D07909340078093E9
:103B30003F0723E530E0309332072093310730937D
:103B4000340720933307909336078093350790937B
:103B5000380780933707109242071092410710925E
:103B600044071092430780E490E0909346078093C7
:103B70004507909348078093470710924A07109291
:103B8000490710924C0710924B0782E490E0909303
:103B90004E0780934D079093500780934F070895E9
:103BA0004532510520F4423010F00C94DB1DFB012E
:103BB0001082CB010895BB274A3031F4992322F4B7
:103BC000BDE2909581959F4F0C94F21D45325105B1
:103BD00020F4423010F00C94F11DFB011082CB0157
:103BE0000895BB27FB015527AA27880F991FAA1FF5
:103BF000A41710F0A41B83955051B9F7A05DAA3308
:103C000008F0A95DA193009779F7B111B1931192D2
:103C1000CB010C940B1EDC01FC01672F7191772303
:103C2000E1F7329704C07C916D9370836291AE1777
:103C3000BF07C8F30895F999FECF92BD81BDF89AE8
:103C4000992780B50895262FF999FECF1FBA92BD06
:103C500081BD20BD0FB6F894FA9AF99A0FBE01966D
:103C60000895052E97FB1EF400940E94481E57FDF0
:103C700007D00E94921E07FC03D04EF40C94481EFD
:103C800050954095309521953F4F4F4F5F4F089588
:103C900090958095709561957F4F8F4F9F4F0895B8
:103CA0000E94B41EA59F900DB49F900DA49F800DFF
:103CB000911D112408952F923F924F925F926F921F
:103CC0007F928F929F92AF92BF92CF92DF92EF92AC
:103CD000FF920F931F93CF93DF93CDB7DEB7CA1B2D
:103CE000DB0B0FB6F894DEBF0FBECDBF09942A8858
:103CF000398848885F846E847D848C849B84AA8400
:103D0000B984C884DF80EE80FD800C811B81AA818C
:103D1000B981CE0FD11D0FB6F894DEBF0FBECDBF57
:103D2000ED010895A1E21A2EAA1BBB1BFD010DC0D7
:103D3000AA1FBB1FEE1FFF1FA217B307E407F5075B
:103D400020F0A21BB30BE40BF50B661F771F881F37
:103D5000991F1A9469F760957095809590959B01CD
:103D6000AC01BD01CF010895A29FB001B39FC00176
:103D7000A39F700D811D1124911DB29F700D811D97
:103D80001124911D0895AA1BBB1B51E107C0AA1F56
:103D9000BB1FA617B70710F0A61BB70B881F991FEC
:103DA0005A95A9F780959095BC01CD010895EE0F25
:103DB000FF1F0590F491E02D0994CF93DF9382309B
:103DC000910510F482E090E0E0919207F091930762
:103DD00020E030E0C0E0D0E0309711F14081518127
:103DE00048175907C0F04817590761F48281938139
:103DF000209719F09B838A832BC09093930780931D
:103E0000920726C02115310519F04217530718F4FF
:103E10009A01BE01DF01EF010280F381E02DDCCFCA
:103E20002115310509F1281B390B2430310590F497
:103E300012968D919C9113976115710521F0FB01EC
:103E40009383828304C09093930780939207FD012C
:103E5000329644C0FD01E20FF31F819391932250EB
:103E600031092D933C933AC02091900730919107EE
:103E7000232B41F420910F013091100130939107D1
:103E80002093900720910D0130910E0121153105ED
:103E900041F42DB73EB74091110150911201241BFE
:103EA000350BE0919007F0919107E217F307A0F42A
:103EB0002E1B3F0B2817390778F0AC014E5F5F4F80
:103EC0002417350748F04E0F5F1F5093910740931A
:103ED00090078193919302C0E0E0F0E0CF01DF9181
:103EE000CF9108950F931F93CF93DF93009709F419
:103EF0008CC0FC01329713821282009192071091BC
:103F000093070115110581F420813181820F931FE0
:103F100020919007309191072817390779F5F09390
:103F20009107E093900771C0D80140E050E0AE17D0
:103F3000BF0750F412962D913C911397AD012115B6
:103F4000310509F1D901F3CF9D01DA0133832283D1
:103F500060817181860F971F8217930769F4EC01C6
:103F600028813981260F371F2E5F3F4F31832083F1
:103F70008A819B8193838283452B29F4F093930755
:103F8000E093920742C01396FC93EE931297ED01D3
:103F9000499159919E01240F351FE217F30771F4DF
:103FA00080819181840F951F029611969C938E9328
:103FB0008281938113969C938E931297E0E0F0E0B8
:103FC000D80112968D919C911397009719F0F801E2
:103FD0008C01F6CF8D919C9198012E5F3F4F820FFF
:103FE000931F20919007309191072817390769F4A2
:103FF000309729F4109293071092920702C013820F
:1040000012821093910700939007DF91CF911F9137
:104010000F910895A0E0B0E0E0E1F0E20C945F1EA3
:10402000EC01009721F4CB010E94DD1EB8C0FC0119
:10403000E60FF71F9C0122503109E217F30708F43D
:10404000ACC0D9010D911C91119706171707B0F05C
:104050000530110508F49FC0C8010497861797071B
:1040600008F499C002501109061B170B0193119314
:104070006D937C93CF010E94721F8DC05B01A01ACB
:10408000B10A4C01800E911EA0919207B091930746
:1040900040E050E0E12CF12C109709F44AC0A8153B
:1040A000B905D1F56D907C901197630182E0C80E3F
:1040B000D11CCA14DB0480F1A3014A195B096A010F
:1040C00082E0C80ED11C1296BC9012971396AC9148
:1040D000B5E0CB16D10440F0B282A3835183408374
:1040E000D9016D937C930AC00E5F1F4FC301800FEF
:1040F000911FF90191838083EB2DFA2FE114F104D4
:1041000031F0D7011396FC93EE93129744C0F093CD
:104110009307E09392073FC08D919C9111974817A8
:10412000590708F4AC017D0112960D90BC91A02DA9
:10413000B3CF809190079091910788159905E1F48C
:1041400046175707C8F480910D0190910E01009712
:1041500041F48DB79EB74091110150911201841B1B
:10416000950BE817F907C8F4F0939107E0939007CF
:10417000F901718360830FC0CB010E94DD1E7C01B9
:10418000009759F0A801BE010E94D920CE010E94DB
:10419000721FC70104C0CE0102C080E090E0CDB71D
:1041A000DEB7EEE00C947B1E81E090E0F8940C9476
:1041B000E920FB01DC0102C001900D92415050400A
:1041C000D8F70895FB01DC0101900D920020E1F782
:0641D0000895F894FFCFF2
:1041D60001FFFFFFFF00E100000000000000009467
:1041E60007800000C1808100000000000000DD049F
:1041F600810A6E06F304FE049606720600000000AD
:1042060091057D05A4056F0576057305700500000B
:104216000000A205466F756E642064617920200057
:1042260020617420726567697374657220706F739C
:1042360020000D0A0073617665416E6451756974DC
:10424600005361766520646179200020746F2065D3
:1042560078697374696E67207265676973746572CD
:1042660020706F73200020746F206672656520725F
:104276006567697374657220706F73200063686187
:104286006E6765204461746520746F20002C000001
:00000001FF
